:0600000000F012EF00F019
:04000800DBEF0AF030
:1000140007323264D8CFFFF0E0CF0CF0EBEF09F0F9
:1000240000EE4AF04F0EEE6AE806FDE10D6A0C6A36
:0C00340000EE9DF0550EEE6AE806FDE1BE
:1000400000EE99F0140EF66E000EF76E10EE04F04E
:100050000900F5CFEEFFE10602E028EF00F0BEEF69
:020060000FF09F
:100064000650075C0AE3D8B41200D8900232013279
:100074000032062A0650075CF6D7D89005320432BF
:100084000332072A06500718D8B41200F6D7800E98
:10009400051AE96AEA6A53EC09F060EC09F0E0DF5A
:1000A40008B017D808A207D0031E041E051E000EB0
:1000B400032A04220522035000260450012205507D
:1000C4000222086A02AE7BEF09F003D808807BEFB6
:1000D40009F0001E011E021E000E002A0122022247
:1000E4001200026A016A006AE950EA1006E002C0DE
:1000F400EDFF01C0EDFF00C0EFFF000C01050000A3
:1001040002000400060008000B000D000F0011009F
:1001140013001500170019001C001E002000220007
:100124002400260028002B002D002F00310033006E
:10013400350037003A003C003E00400042004400D5
:10014400470049004B004D004F0051005400560039
:1001540058005A005C005F0061006300650067009E
:100164006A006C006E007000720075007700790000
:100174007B007D00800082008400860088008B0064
:100184008D008F0091009300960098009A009C00C7
:100194009E00A100A300A500A700AA00AC00AE0029
:1001A400B000B200B500B700B900BB00BD00C0008C
:0C01B400C200C400C600C900CB00CD0092
:1001C000CF00D100D400D600D800DA00DC00DF0078
:1001D000E100E300E500E700EA00EC00EE00F000DB
:1001E000F200F500F700F900FB00FD00FF0002013E
:1001F0000401060108010A010D010F01110113019B
:10020000150117011A011C011E0120012201240100
:10021000270129012B012D012F0131013401360164
:1002200038013A013C013E014001430145014701CB
:1002300049014B014D015001520154015601580131
:100240005A015C015E016101630165016701690199
:100250006B016D01700172017401760178017A0100
:100260007C017E01810183018501870189018B0168
:100270008D018F0192019401960198019A019C01D0
:100280009E01A001A301A501A701A901AB01AD0138
:10029000AF01B101B401B601B801BA01BC01BE01A0
:1002A000C001C301C501C701C901CB01CD01CF0107
:1002B000D101D401D601D801DA01DC01DE01E0016F
:1002C000E301E501E701E901EB01ED01EF01F201D5
:1002D000F401F601F801FA01FC01FF010102030239
:1002E0000502070209020B020E021002120214029A
:1002F000160218021B021D021F02210223022602FF
:1003000028022A022C022E02300233023502370262
:1003100039023B023D0240024202440246024802C8
:100320004B024D024F0251025302560258025A022A
:100330005C025E02600263026502670269026B0290
:100340006E02700272027402760279027B027D02F2
:100350007F0282028402860288028A028D028F0254
:1003600091029302950298029A029C029E02A002B8
:10037000A302A502A702A902AC02AE02B002B20219
:10038000B402B702B902BB02BD02BF02C202C4027C
:10039000C602C802CB02CD02CF02D102D302D602DE
:1003A000D802DA02DC02DF02E102E302E502E8023F
:1003B000EA02EC02EE02F002F302F502F702F902A1
:1010DE00001E011E021E031E000E002A0122022205
:1010EE0003221200046E042A0406D8B4000CD89011
:1010FE000332023201320032F7D7026A01BE020613
:10110E000250036E9FEF08F0026A036AA5EF08F023
:10111E00036A026A016A006AE950EA1008E003C035
:10112E00EDFF02C0EDFF01C0EDFF00C0EFFF000CB0
:10113E0003AE04D008806FEC08F001D0086A8E0E62
:10114E00066EE96AEA6A0352D8B47BEF09F0D890CA
:10115E000332023201320032062AF5D7E96AEA6A10
:10116E0053EC09F0036A820E062606BE5CEF09F008
:10117E00F00E062606BE11D0180E065C02E35CEFDA
:10118E0009F0065204E108B06FEC08F012000606F2
:10119E000036013602360336F4D7D89002320132C9
:1011AE000032063EFAD7EFD7896A080E8A6E330EE2
:1011BE00926EF50E936E010EC26E7C0EC16EAD0E6A
:1011CE00C06E9F9C9E9C9D8C200EAC6E900EAB6E46
:1011DE000C0EAF6E9F9A9F989D8A840ED56EFD0E53
:1011EE00D76E950ED66EF194F294F28A800ECD6E75
:1011FE00FD0ECF6EA70ECE6E9F809E909D80F18CC1
:10120E00F292F288F198F09EF092F088D08E120051
:10121E00E96AEA6A0050086E0150096E02500A6EC1
:10122E0003500B6E026A036A08500402F3CF00F0FB
:10123E00F4CF01F008500502F3500126F4500222BB
:10124E0009500402F3500126F4500222D8B0032AAA
:10125E0008500602F3500226F450032209500502EC
:10126E00F3500226F45003220A500402F3500226D1
:10127E00F450032208500702F350032609500602C9
:10128E00F35003260A500502F35003260B500402B6
:10129E00F350032693EF08F0086A01340234066E09
:1012AE0004E00836026A018E1200006A016A026AC0
:1012BE00000C089204340534076E05E0D8B008829D
:1012CE00056A048E1200076A036A046A056A120030
:1012DE0006480D800650E9E0019E08320630026E87
:1012EE00D8B0018E76EF00F0065220E0025010E0EA
:1012FE00020403E1002A01220222D89002320132B6
:10130E000032062AF1E10250EFE00DA60D92F0D761
:10131E000050011002100AE001BEDAD7062E02D0EC
:10132E000D82DAD7D89000360136F6D773EF00F07B
:10133E00E96AEA6A53EC09F060EC09F0096A0A6A94
:10134E000B6A070E056ED8900432033206E3005086
:10135E00092601500A2202500B22D890003601367F
:10136E000236052EF0D7090E056E04D0D8900B323A
:10137E000A320932D8900432033206E300500926AD
:10138E0001500A2202500B22052EF0D70830081AFF
:10139E000950006E0A50016E0B50026E0D960DB282
:1013AE000D8606520AE0075008E00626860E07E371
:1013BE00065ED8B00D807BEF09F073EF00F0065E8D
:1013CE00D8A00D827BEF09F0E8CFFEF0E9CFFDF05B
:1013DE00EACFFCF004C0FBF003C0FAF002C0F9F053
:1013EE0001C0F8F000C0F7F0F7CFF6F0F6CFF5F049
:1013FE00F5CFF4F0F4CFF3F0F3CFF2F0F2B4F2AAAB
:10140E000CD0F294FD0ED76E950ED66EB0839C2F37
:10141E0004D0640EE8CF9CF0B0859EBA9DAA16D07B
:10142E00ABA403D0AECFB1F011D0AECFB1F0A82B9C
:10143E001D0EA86501D0A86BA8C0E8FF00EEB2F0A3
:10144E00E926000EEA22B1C0EFFFB0879EB89DA834
:10145E0014D09FC0E8FFA9190FE09FC0E8FF00EE6F
:10146E00D0F0E926000EEA22EF50AD6E9F2B1D0E36
:10147E009F6503D09F6B01D09D989EBC9DAC6CD098
:10148E009E9CC350F66EF76AC450F712A2C0E8FFD6
:10149E00040D5C0EF324E96E000EF420EA6EF65095
:1014AE00EE26F750EE22000EEE22ED22ED52ED5218
:1014BE00A22B010EA26542D0A26BA2C000F0016A5F
:1014CE000050000FF66E0150F76E010EF722080065
:1014DE00F550C26EA52B3F0EA5653ED0A56B060E30
:1014EE005CC000F05DC001F05EC002F05FC003F0B2
:1014FE0079EC08F000C054F001C055F0060E00EE75
:10150E0060F0EECF00F0EECF01F0EECF02F0EECFB6
:10151E0003F079EC08F000EE56F000C0EEFF01C0CB
:10152E00EDFF00EE5CF0EE6AEE6AEE6AEE6A00EE39
:10153E0060F0EE6AEE6AEE6AED6A0ED0A2C000F0BE
:10154E00016A0050000FF66E0150F76E010EF72281
:10155E000800F550C26EC282F0B2F0A806D0F0922A
:10156E00A42BC80EA46501D0AE83F2C0F3FFF3C066
:10157E00F4FFF4C0F5FFF5C0F6FFF6C0F7FFF7C0B5
:10158E0000F0F8C001F0F9C002F0FAC003F0FBC0A1
:10159E0004F0FCC0EAFFFDC0E9FFFEC0E8FF0CC08E
:1015AE00E0FFFFC0D8FF10009EB09DA007D0C28202
:1015BE009E90CD90FD0ECF6EA70ECE6EF2B2F2A81B
:1015CE001100CD80F292A32B630EA36501D0A36B05
:1015DE00AAC0E8FFA36103D08A96A46B11008A8685
:1015EE001100D96EF29EA9C0E8FF00EED0F0E926F8
:1015FE00000EEA22D9CFEFFFA92B1D0EA96501D04F
:10160E00A96BACA20ED09FC0E8FF00EED0F0E92689
:10161E00000EEA22EF50AD6E9F2B1D0E9F6501D07E
:10162E009F6B9D88F28E1200F29E9E2B1D0E9E6564
:10163E0001D09E6BA8C0E8FF9E6301D0B097F28EDA
:10164E009EC0E8FF00EEB2F0E926000EEA22EF504F
:10165E001200B0A71200E8DFE8CFF0F0F0C000F003
:10166E00002803E1040EAB1B0DD0ABA50BD0AB8154
:10167E00AB93AB95210EE8CFEFF0EE6B670E646F78
:10168E00000E656FABB51200ABA116D0EF07EF29B8
:10169E000CE0EFC0E8FF1E0A0FE11E0EF06502D04F
:1016AE00AB910AD0F0C0EFF007D0AB91AB83F0C096
:1016BE00E8FFEE6301D0AB87ABB3120064C0E9FF65
:1016CE0065C0EAFFF0C0EFFF642B000E6523F0C08B
:1016DE00E8FFEE271200E16AFF0E83DF67C0E8FF26
:1016EE0080DF68C0E8FF7DDF69C0E8FF7ADF67C092
:1016FE00E8FFE12668C0E8FFE12669C0E8FFE126C1
:10170E00F36A69C0E8FFF35C1EE2F35000EE6AF084
:10171E00E926000EEA22EF50E126F35000EE6AF0C1
:10172E00E926000EEA22EF505CDFF35000EE6AF07D
:10173E00E926000EEA22EF50006E002802E1FF0EAD
:10174E0050DFF32ADED7E1504CDFE128D8A4120097
:10175E00FF0E47D7ABA71200AB97A1D000EE69F0F2
:10176E00EF50010E01E097D0E8CF6BF0E8CF6CF0B0
:10177E00030E42D000EE69F0EF5001E08BD050C066
:10178E006AF051C06BF0ACC06CF058C06DF059C02F
:10179E006EF05AC06FF05BC070F0070E2DD000EEE9
:1017AE0069F0EF5077E1AEC06AF0010E25D069C046
:1017BE00E8FF070A6FE16AC050F06BC051F06CC0D1
:1017CE00ACF06DC058F06EC059F06FC05AF070C0DA
:1017DE005BF0696BB08185D069C000F000045AE1FE
:1017EE006AC0AFF055D000EE69F0EF5053E14CC037
:1017FE006AF04DC06BF0020EE8CF69F072D069C08E
:10180E00E8FF020A47E16AC052F06BC053F040D0C5
:10181E0069C000F000043EE16AC0ADF0ADC0E8FF63
:10182E00A65DE8CFA7F0A7C0E8FFA02754C0A1F09F
:10183E00410EA06502D0E8CFA0F0230EA06102D029
:10184E00E8CFA0F01E0EA16502D0E8CFA1F00A0EDF
:10185E00A1611DD0E8CFA1F01AD069C0E8FF020A3D
:10186E0019E16AC04EF06BC04FF012D000EE69F075
:10187E00EF5010E14EC06AF04FC06BF0BCD769C09C
:10188E00E8FF020A07E16AC04EF06BC04FF0B08964
:10189E00696B27D0010EE8CF69F0030E20D068C027
:1018AE00E8FF010A01E15AD7030A01E163D7010AF1
:1018BE0001E175D7070A01E17AD7010A8DE0030A23
:1018CE0092E0010A9CE00F0AA3E0010AC6E0030AB7
:1018DE00CDE0010AD4E0010EE8CF69F0020EE8CFA8
:1018EE006AF0F9DE040012009300010E945D5F0EA3
:1018FE00D8B4935D04E35E0E936F010E946FD8908F
:10190E009335006E9435016E0050020FF66E015045
:10191E00F76E010EF7220900F5CF00F00900F5CFA2
:10192E0001F012009300BE0EF66E030EF76E090064
:10193E00F5CF00F00900F5CF01F09451015C02E102
:10194E009351005C05E25E0E006E010E016E1200F8
:10195E00976B986B5E0E956F010E966F9851965D14
:10196E0002E19751955DD8A0120097C000F098C083
:10197E0001F09551002696510122D8900130F46E57
:10198E000030F36ED890F334006EF434016E0050D4
:10199E00020FF66E0150F76E010EF7220900F5CF19
:1019AE0000F00900F5CF01F00150945D02E1005006
:1019BE00935D5DE2FF0EF324956FFF0EF420966F9C
:1019CE00D8909535006E9635016E0050020FF66E6A
:1019DE000150F76E010EF7220900F5CF00F0090055
:1019EE00F5CF01F09451015C02E19351005CB6E237
:1019FE00D8909535006E9635016E0050020FF66E3A
:101A0E000150F76E010EF7220900F5CF02F0090022
:101A1E00F5CF03F0D890F334006EF434016E00501D
:101A2E00020FF66E0150F76E010EF7220900F5CF88
:101A3E0000F00900F5CF01F002500024F66E0350BD
:101A4E000120F76ED890F730016EF630006E94518B
:101A5E00015C02E19351005C05E395C000F096C075
:101A6E0001F01200F3CF00F0F4CF01F01200D89085
:101A7E00F334006EF434016E0050020FF66E015016
:101A8E00F76E010EF7220900F5CF00F00900F5CF31
:101A9E0001F09451015C02E19351005C5DE2F32888
:101AAE00976F000EF420986FD8909735006E98358A
:101ABE00016E0050020FF66E0150F76E010EF72206
:101ACE000900F5CF00F00900F5CF01F00150945D4B
:101ADE0002E10050935D01E341D7D8909735006E37
:101AEE009835016E0050020FF66E0150F76E010E22
:101AFE00F7220900F5CF02F00900F5CF03F0D890D8
:101B0E00F334006EF434016E0050020FF66E015085
:101B1E00F76E010EF7220900F5CF00F00900F5CFA0
:101B2E0001F002500024F66E03500120F76ED8909B
:101B3E00F730016EF630006E9451015C02E1935164
:101B4E00005C05E297C000F098C001F01200F3CFE0
:101B5E0000F0F4CF01F01200F3CF00F0F4CF01F05B
:101B6E001200E10E006EFA0E016E3E0E026E00C005
:101B7E0090F001C091F002C092F000EE56F0EECF60
:101B8E0000F0EDCF01F08BEC08F090C003F091C0A7
:101B9E0004F092C005F09FEC09F0B5EC08F0A0C07F
:101BAE0002F00250005CE8CFA6F054C000F055C021
:101BBE0001F0A1C002F0036A0150035C02E1005083
:101BCE00025C45E2A1C0E8FF54C000F055C001F030
:101BDE00005CF66E0150D8A00104F76E4EC000F006
:101BEE004FC001F00050046E0150056E066A076A80
:101BFE00F6CF00F0F7CF01F0026A036A0FEC09F09E
:101C0E0000C08CF001C08DF002C08EF003C08FF0CA
:101C1E008DC08CF08EC08DF08FC08EF08F6B8CC00F
:101C2E008AF08DC08BF0A6C093F0946B5EDE00C080
:101C3E0088F001C089F088518A25936F89518B21D4
:101C4E00946F71DE00C04CF001C04DF01200A6C0C2
:101C5E004CF04D6B12008800A96E8851A86EA69CA0
:101C6E00A69EF29EA684550EA76EAA0EA76EA682FB
:101C7E00F28EA1A8FED7A198A6941200A69CA96EDA
:101C8E00A69EA680A8501200500EE16E000EE26EC7
:101C9E00E750886F000EE0DFE652E750886F010EC6
:101CAE00DBDFAC0EE16E000EE26EE750886F020EC7
:101CBE00D3DF580EE16E000EE26EE750886F030E12
:101CCE00CBDFE652E750886F040EC6DFE652E750D0
:101CDE00886F050EC1DFE652E750886F060EBCD73F
:101CEE00A0C088F0070EB8DFA1C088F0080EB4DFE0
:101CFE004E0EE16E000EE26EE750886F090EACDFFD
:101D0E00E652E750886F0A0EA7D7500EE16E000E0E
:101D1E00E26E000EB3DFE76EE652010EAFDFE76E46
:101D2E00AC0EE16E000EE26E020EA8DFE76E580EEC
:101D3E00E16E000EE26E030EA1DFE76EE652040EB8
:101D4E009DDFE76EE652050E99DFE76EE652060E50
:101D5E0095DFE76E010E515D2D0ED8B4505D06E293
:101D6E00000E515D1E0ED8B4505D04E21E0E506F73
:101D7E00516BB0810A0EAC6501D003D0010EAC617F
:101D8E0004D0010EE8CFACF0B08110EE5BF0000E87
:101D9E00E55C08E1010EE55C05E1510EE55C02E152
:101DAE00810EE75CD8A0120010EE58F0E66AE66AE3
:101DBE00E66AE66AB0811200070E60DFE8CFA0F097
:101DCE00080E5CDFE8CFA1F04E0EE16E000EE26E63
:101DDE00090E54DFE76EE6520A0E50DFE76E410E33
:101DEE00A06501D003D0230EA06104D0320EE8CF3F
:101DFE00A0F0B0891E0EA16501D003D00A0EA1611C
:101E0E0004D0140EE8CFA1F0B089010E4F5D510E33
:101E1E00D8B44E5D07E2000E4F5DB00ED8B44E5DE5
:101E2E00D8B012004E6B010E4F6FB089120052C027
:101E3E0000F053C001F04CC0E8FF005C026E4DC0D4
:101E4E00E8FF0158036E0350800A800F140ED8B4B9
:101E5E00025C1AE2000E535DFB0ED8B4525D02E333
:101E6E005A0E13D0000E535D970ED8B4525D02E396
:101E7E00500E0BD0000E535D650ED8B4525D02E3CA
:101E8E00460E03D0320E01D0640ED96E52C000F051
:101E9E0053C001F04CC0E8FF005CF66E4DC0E8FF89
:101EAE000158F76E4AC000F04BC001F084EC08F008
:101EBE0000C08AF001C08BF002C08CF03D0E006EA7
:101ECE008A0E016E3F0E026E00C08DF001C08EF0C4
:101EDE0002C08FF0F6CF00F0F7CF01F084EC08F0DF
:101EEE008DC003F08EC004F08FC005F09FEC09F09A
:101EFE008AC003F08BC004F08CC005F049EC00F0F2
:101F0E00B5EC08F0D89000360136D8900036013680
:101F1E00D8900036013600C088F001C089F09DC00F
:101F2E00E8FF8825F36E000E8921F46EF4AE02D020
:101F3E00AA6B15D0D9CF00F0016A00BE0106015080
:101F4E00800A026EF450800A025C02E1F350005CDB
:101F5E0004E2D9CFAAF0AE8703D0F3CFAAF0AE97A2
:101F6E00AAC09DF0F6CF4AF0F7CF4BF01200DBEC93
:101F7E0008F0F28EF28CC9DE1FDF30EC0BF0B1EC04
:101F8E000BF0B0A314D0B09380B804D09A2F05D024
:101F9E00AE8103D0320EE8CF9AF081AE04D09B2FE3
:101FAE0006D0AE8504D0320EE8CF9BF0AE95B0A52C
:101FBE000CD0B095B8EC0DF0AFA307D099079929C6
:101FCE0004E1070EE8CF99F032DFB0A102D0B09154
:101FDE005BDEB0A902D0B09983DEAFA102D08986B4
:101FEE0001D08996AFA302D08984C7D78994996B03
:021FFE00C4D746
:020000040030CA
:0E000000FF32F2F5FF7FFBFFFFFFFFFFFFFF68
:00000001FF
